S01A000064656D6F70726F675F73746D3332663035312E7372656399
S3150800200000200020113300086133000861330008FE
S3150800201000000000000000000000000000000000B2
S315080020200000000000000000000000006133000806
S31508002030000000000000000061330008913300082A
S315080020406133000861330008613300086133000812
S315080020506133000861330008613300086133000802
S3150800206061330008613300086133000861330008F2
S3150800207061330008613300086133000861330008E2
S31508002080613300086133000800000000613300086E
S3150800209061330008613300086133000861330008C2
S315080020A061330008613300086133000861330008B2
S315080020B061330008000000006133000800000000DA
S309080020C0EE11AA5510
S315080020C410B5064C2378002B07D1054B002B02D0FC
S315080020D4044800E000BF0123237010BDC40000209B
S315080020E400000000E4330008044B10B5002B03D0AD
S315080020F40349044800E000BF10BDC04600000000C4
S31508002104C8000020E4330008002243088B4274D335
S3150800211403098B425FD3030A8B4244D3030B8B42D6
S3150800212428D3030C8B420DD3FF22090212BA030CDF
S315080021348B4202D31212090265D0030B8B4219D3C0
S3150800214400E0090AC30B8B4201D3CB03C01A5241E0
S31508002154830B8B4201D38B03C01A5241430B8B4228
S3150800216401D34B03C01A5241030B8B4201D30B0311
S31508002174C01A5241C30A8B4201D3CB02C01A524138
S31508002184830A8B4201D38B02C01A5241430A8B42FB
S3150800219401D34B02C01A5241030A8B4201D30B02E4
S315080021A4C01A5241CDD2C3098B4201D3CB01C01AFE
S315080021B4524183098B4201D38B01C01A5241430908
S315080021C48B4201D34B01C01A524103098B4201D3F6
S315080021D40B01C01A5241C3088B4201D3CB00C01A63
S315080021E4524183088B4201D38B00C01A52414308DB
S315080021F48B4201D34B00C01A5241411A00D2014600
S31508002204524110467047FFE701B5002000F006F872
S3150800221402BDC0460029F7D076E770477047C04626
S3150800222410B50948094B0360E1231B0243600023E8
S315080022348360C36003610C2242618361C3610362E4
S31508002244436200F06DFF10BDE0000020004400402A
S3150800225410B5010000230122044800F09DFE002861
S3150800226401D0002010BD0130FCE7C046E000002084
S3150800227410B5FFF7D5FF10BDBFF34F8F034A044BC4
S31508002284DA60BFF34F8FC046FDE7C0460400FA057F
S3150800229400ED00E010B5214B1B78002B16D1204821
S315080022A4FFF7D6FF012800D010BD1D4B1B78013B54
S315080022B4DBB23F2BF8D801F065F81A4B18600122F7
S315080022C4164B1A700022184B1A70EDE7164B1B783A
S315080022D401331348C018FFF7BBFF01280AD001F0E1
S315080022E451F8104B1B6864339842DDD900220B4B16
S315080022F41A70D9E70C4A13780133DBB21370084A0B
S3150800230412789342D0D10021044A1170044A5278B3
S31508002314FF2AC9D1022BC7D1FFF7AEFF91010020CE
S3150800232450010020940100209201002010B5FFF707
S31508002334B1FF10BD10B5002280218900014800F0C4
S3150800234487F910BD0008004810B501F01BF8040011
S315080023540F4B1B68C31AF422FF3293420ED90D4B56
S315080023641B78002B0BD1F33AFF3A0A4B1A708021DB
S315080023748900094800F06CF9054B1C6010BD002261
S31508002384044B1A7080218900034800F061F9F3E7C9
S315080023949C010020980100200008004810B504009C
S315080023A400F062FCFA218900FFF7AEFE00F058F847
S315080023B4002221000120404200F020F8002010BD30
S315080023C410B5064A136810210B4313600020FFF763
S315080023D4E5FF00F047FF002010BDC046002002407C
S315080023E4024A1368013313607047C046A0010020EF
S315080023F4014B18687047C046A001002070B5002834
S3150800240411DB8308144DC0339B005C59032210402A
S31508002414C000FC3216008640B44389010A40824053
S3150800242422435A5170BDC0B20F230340083B9B0890
S3150800243406339B00094A944663445D6803221040A8
S31508002444C000FF2422008240954389010C40844041
S315080024542C435C60E6E7C04600E100E000ED00E0DE
S3150800246401380A4B98420FD8094A50600948036A4A
S315080024741B021B0AC02109060B430362002393604F
S3150800248407331360002070470120FCE7FFFFFF00B5
S3150800249410E000E000ED00E0042805D0054A1368C2
S315080024A404218B4313607047024A136804210B43C3
S315080024B41360F8E710E000E0704710B5FFF7FCFF7B
S315080024C410BD0000F0B5C64600B582B000237EE014
S315080024D4DF080837BF003E5807251D40AD000F2406
S315080024E4AC40A6430C69AC40250035433D507EE01C
S315080024F4856864462540CE68BE4035438560456890
S315080025042C004546AC434D682E09012535409D40AF
S315080025142C434460C46865462C408D68BD402C43F2
S31508002524C4604C68E40051D5434DAE690124264382
S31508002534AE61AD692C400194019C9C08A51CAD00B4
S315080025443E4EAE5903251D40AD000F27AF40BE438E
S315080025549027FF05B84265D0394FB84264D0394F41
S31508002564B84263D0384FB8425AD00527AF403D0029
S3150800257435430234A400314EA551344C2568D4435E
S3150800258426002E404F68FF0301D515432E002F4D14
S315080025942E606D682E0026404F68BF0301D515438B
S315080025A42E002A4D6E60AD682E0026404F68FF0245
S315080025B401D515432E00254DAE60ED682C404E68B6
S315080025C4B60201D52A431400204AD46001330A68A6
S315080025D41400DC402CD001249C40A0462240F5D0AF
S315080025E44D68022D00D173E7122D00D170E70668F5
S315080025F45F0003252C00BC40E443A44626404C68EF
S315080026042540BD40354305604D686E1E012E00D831
S315080026146EE7112D00D16BE7122D00D07AE767E734
S315080026240327A3E70027A1E701279FE702279DE7DA
S3150800263402B004BC9046F0BD001002400000014000
S315080026440004004800080048000C00480004014043
S31508002654002A01D1816270478161FCE770B582B0B6
S3150800266404000368DB0736D5C14B5A680C231340AC
S31508002674042B28D0BE4B5A680C231340082B1ED0B3
S315080026846368012B4BD0002B50D1B94B1A68B94952
S315080026940A401A601A68B8490A401A606368002B27
S315080026A45CD0FFF7A5FE0500B14B1B689B0312D44B
S315080026B4FFF79EFE401B6428F6D90320EAE1AC4BDB
S315080026C45B68DB03DCD5AA4B1B689B0303D56368ED
S315080026D4002B00D1DBE123689B0762D5A44B5B681A
S315080026E40C221A424CD0A24B5A680C231340082BCE
S315080026F442D0E368002B76D09D4A136801210B4328
S315080027041360FFF775FE0500994B1B689B0761D498
S31508002714FFF76EFE401B0228F6D90320BAE1944A55
S31508002724116880235B020B431360B7E7052B09D0B6
S315080027348F4B1A688F490A401A601A688E490A40EC
S315080027441A60ABE78A4B19688022D2020A431A60D8
S315080027541968802252020A431A609FE7FFF748FE67
S315080027640500834B1B689B03B5D5FFF741FE401B49
S315080027746428F6D903208DE17D4B5B68DB03B8D466
S315080027847B4B1B689B0704D5E368012B01D001200A
S3150800279480E177490B68F82293432269D2001343F0
S315080027A40B6023681B0744D5E369002B2ED0704AB7
S315080027B4536A01210B435362FFF71AFE05006C4B5B
S315080027C45B6A9B0735D4FFF713FE401B0228F6D92C
S315080027D403205FE166490B68F82293432269D20015
S315080027E413430B60DDE7624A136801218B431360C8
S315080027F4FFF7FEFD05005E4B1B689B07D1D5FFF767
S31508002804F7FD401B0228F6D9032043E1584A536AC8
S3150800281401218B435362FFF7EBFD0500544B5B6ABA
S315080028249B0706D5FFF7E4FD401B0228F6D90320CB
S3150800283430E123685B0775D54D4BDB69DB002ED485
S315080028444B4AD169802040050143D161D3690340CD
S315080028540193019B0125494B1B68DB0521D5A36818
S31508002864012B32D0002B36D1414B1A6A01218A43F7
S315080028741A621A6A03318A431A62A368002B40D083
S31508002884FFF7B6FD06003A4B1B6A9B0748D4FFF7C9
S31508002894AFFD801B3A4B9842F5D90320FAE0002590
S315080028A4D9E7364A116880235B000B431360FFF7A8
S315080028B49FFD0600314B1B68DB05D0D4FFF798FD56
S315080028C4801B6428F6D90320E4E0294A136A012107
S315080028D40B431362D1E7052B09D0254B1A6A01214C
S315080028E48A431A621A6A03318A431A62C5E7204B75
S315080028F41A6A04210A431A621A6A03390A431A62CB
S31508002904BBE7FFF775FD0600194B1B6A9B0707D53E
S31508002914FFF76EFD801B1A4B9842F5D90320B9E0E0
S31508002924012D1ED02368DB065AD56369012B2BD0EB
S31508002934053349D00E4B5A6B04210A435A635A6B22
S3150800294403398A435A63FFF753FD0500084B5B6B4B
S315080029549B0745D5FFF74CFD401B0228F6D90320F3
S3150800296498E0034AD36907490B40D361DAE7C046BE
S3150800297400100240FFFFFEFFFFFFFBFF0070004050
S3150800298488130000FFFFFFEF444B5A6B04210A43E8
S315080029945A635A6B03390A435A63FFF729FD05003C
S315080029A43E4B5B6B9B0706D4FFF722FD401B0228B0
S315080029B4F6D903206EE039494B6BF8229343A26992
S315080029C4D20013434B630BE0344A536B04218B4305
S315080029D45363536BF4318B43A169C9000B435363A7
S315080029E4236A002B55D02D4A51680C220A40082A1E
S315080029F452D0022B12D0294A136829490B40136076
S31508002A04FFF7F6FC0400254B1B689B013DD5FFF731
S31508002A14EFFC001B0228F6D903203BE01F4A136883
S31508002A241F490B401360FFF7E3FC05001B4B1B68AB
S31508002A349B0106D5FFF7DCFC401B0228F6D90320C8
S31508002A4428E0164BDA6A0F218A43E16A0A43DA62F6
S31508002A545A6814490A40A16A606A01430A435A60DB
S31508002A641968802252040A431A60FFF7C1FC04005D
S31508002A740A4B1B689B0106D4FFF7BAFC001B022805
S31508002A84F6D9032006E0002004E0002002E0012035
S31508002A9400E0002002B070BD0120FBE700100240F0
S31508002AA4FFFFFFFEFFFFC2FF30B589B004AA154B2E
S31508002AB4180032C832C2110002680A606A46103326
S31508002AC413CB13C21B6813600F4B5A680C231340AD
S31508002AD4082B13D1910C0733194004A8445C0A49FE
S31508002AE4C96A0B406946C95CD30302D407486043E4
S31508002AF405E00748FFF708FB604300E0044809B00F
S31508002B0430BDC046FC3300080010024000093D00F1
S31508002B1400127A0070B505000C004D4B1A680123A3
S31508002B2413408B420BD24A490B6801229343234331
S31508002B340B600B681A40944201D0012085E02B688B
S31508002B449B0706D5434A5368F0218B43A9680B4370
S31508002B5453602B68DB074CD56B68012B21D0022BFD
S31508002B6425D03C4A1268920700D46FE039494A686E
S31508002B740320824313434B60FFF73AFC06006B6855
S31508002B84012B1AD0022B26D0324B5B680C221A4230
S31508002B942FD0FFF72DFC801B2F4B9842F4D9032026
S31508002BA453E02C4A12689203E0D401204DE0294AE6
S31508002BB412689201DAD4012047E0264B5A680C239E
S31508002BC41340042B15D0FFF713FC801B224B9842A5
S31508002BD4F3D9032039E01F4B5A680C231340082BFA
S31508002BE407D0FFF705FC801B1B4B9842F3D903203B
S31508002BF42BE0174B1A68012313409C420BD2144945
S31508002C040B680122934323430B600B681A409442D2
S31508002C1401D0012019E02B685B0706D50D4A5368D5
S31508002C240E490B40E9680B435360FFF73DFF094B18
S31508002C345A6812090F231340094AD35CD840094B32
S31508002C4418600020FFF7AAFB002070BD0120FCE7EE
S31508002C54002002400010024088130000FFF8FFFF1E
S31508002C641C340008C0000020014B18687047C04691
S31508002C74C000002010B5FFF7F7FF044B5A68120A84
S31508002C8407231340024AD35CD84010BD0010024003
S31508002C942C3400087047000070B504008368026984
S31508002CA4134342691343C269134301680A685F48B8
S31508002CB4024013430B60226853685D490B40E16880
S31508002CC40B435360A369226A134321688A685948E7
S31508002CD4024013438B602568574B9D4220D0574BBF
S31508002CE49D4231D0102380221202E16991422FD0ED
S31508002CF4022B00D17FE000D86FE0042B00D186E0D8
S31508002D04082B00D08FE06168480880231B029C4684
S31508002D146044FFF7F9F90004000CE860002041E07C
S31508002D24474B1A6B03231340012B09D0002B05D0FC
S31508002D34022B07D0032B09D01023D4E70023D2E7AC
S31508002D440423D0E70823CEE70023CCE70223CAE707
S31508002D54022B28D00FD9042B30D0082B3AD163681C
S31508002D64580880235B029C4660446168FFF7CCF9E7
S31508002D7483B200200CE0002B2CD1FFF77BFF400028
S31508002D8463685B08C0186168FFF7BEF983B2002060
S31508002D940F22190091430A005B1007210B401343C5
S31508002DA42268D36070BD63685808264B9C46604405
S31508002DB46168FFF7A9F983B20020E9E7FFF774FE13
S31508002DC4400063685B08C0186168FFF79DF983B221
S31508002DD40020DDE701200023DAE7002B23D1FFF7E3
S31508002DE449FF61684B08C018FFF78EF90004000C08
S31508002DF4E8600020D6E761684808134B9C4660449F
S31508002E04FFF782F90004000CE8600020CAE7FFF720
S31508002E144BFE61684B08C018FFF776F90004000CEE
S31508002E24E8600020BEE70120BCE7C046F369FFFF5F
S31508002E34FFCFFFFFFFF4FFFF0038014000440040C6
S31508002E44001002400024F40000127A00436ADB07EB
S31508002E5406D5026853682C490B40816A0B435360B4
S31508002E64436A9B0706D50268536828490B40C16A1A
S31508002E740B435360436A5B0706D5026853682449C3
S31508002E840B40016B0B435360436A1B0706D5026864
S31508002E94536820490B40416B0B435360436ADB0676
S31508002EA406D5026893681C490B40816B0B439360F3
S31508002EB4436A9B0606D50268936818490B40C16B9A
S31508002EC40B439360436A5B060BD50268536814493F
S31508002ED40B40016C0B43536080235B03026C9A42DC
S31508002EE40AD0436A1B0606D5026853680D490B4087
S31508002EF4816C0B4353607047026853680A490B4058
S31508002F04416C0B435360ECE7FFFFFDFFFFFFFEFF39
S31508002F14FFFFFBFFFF7FFFFFFFEFFFFFFFDFFFFF63
S31508002F24FFFFEFFFFFFFF7FFFFFF9FFFF0B5C64662
S31508002F3400B505000F0016009846069C2B68DB6949
S31508002F443A009A4313005A425341B3421ED1631CB2
S31508002F54F4D0002C05D0FFF74BFA4346C01A844236
S31508002F64ECD22A6813680B490B4013602A689368E5
S31508002F74A331FF318B43936020236922AB5401327A
S31508002F84AB5400224833EA54032000E0002004BC72
S31508002F949046F0BD5FFEFFFFF0B585B004000F0054
S31508002FA416001D006A23C35C202B02D0022005B03C
S31508002FB4F0BD002970D0002A70D080235B01826896
S31508002FC49A4205D06823E35C012B08D10220EEE778
S31508002FD40369002BF6D1CB07F4D50120E7E70122D4
S31508002FE46823E2540023E36621326A33E254FFF786
S31508002FF4FFF903905823E6520233E652A368802267
S31508003004520193420AD0002B05D12369002B10D113
S31508003014FF225C33E2525C23E65A14E02369002B50
S3150800302403D1204A5C33E252F5E7FF225C23E252DD
S31508003034F1E77F225C23E252EDE723689B8CF2B228
S3150800304413403B7001375A23E35A9BB2002B1BD01B
S315080030545A22A35A013B9BB2A3520095039B002212
S3150800306420212000FFF762FF002819D180235B0185
S31508003074A2689A42E1D12369002BDED123689B8C8E
S3150800308433403B800237DEE720226A33E2540022CB
S31508003094023BE25400208AE7012088E7012086E7FC
S315080030A4032084E7FF01000030B583B00400002341
S315080030B4C366FFF79DF905002368174A93420AD0A9
S315080030C420236922A3540132A35400224833E2542C
S315080030D4002003B030BD1B681B0710D423681B6887
S315080030E45B07EDD50D4B00932B0000228021C90305
S315080030F42000FFF71BFF0028E2D00320E9E7074B6F
S31508003104009303000022802189032000FFF70EFFA5
S315080031140028E3D00320DCE700380140FFFFFF0165
S3150800312410B5041E30D06923C35C002B22D0242298
S315080031346923E2542268136801218B431360200033
S31508003144FFF7AAFD012814D0636A002B18D1226858
S3150800315453680E490B405360226893682A218B43AF
S3150800316493602268136829390B4313602000FFF71C
S315080031749BFF10BD00226833C254FFF78BFDD6E7C8
S315080031842000FFF763FEE2E70120F2E7FFB7FFFF3F
S31508003194114B1A6801210A431A605A680F480240FB
S315080031A45A601A680E4802401A601A680D480240A6
S315080031B41A605A680C4802405A60DA6A0F20824339
S315080031C4DA621A6B094802401A635A6B8A435A63CD
S315080031D400229A607047C046001002400CB8FFF8F7
S315080031E4FFFFF6FEFFFFFBFFFFFFC0FFACFEFFFF7E
S315080031F400B591B00123049304330593033B0C9360
S3150800320480235B020D9380235B030E9300230F93A5
S3150800321404A8FFF723FA002800D0FEE70723009343
S31508003224053B019300230293039301216846FFF7A4
S3150800323471FC002800D0FEE711B000BD10B5FFF7F9
S31508003244BFF8FFF7D5FFFFF775F800F088F810BD4B
S3150800325410B5FFF7F3FFFFF70BF8FFF775F8FFF75D
S3150800326465F8FAE730B58BB0264B9A6901242243F0
S315080032749A619A6922400192019A596980229202B6
S315080032841143596159691140029102995869802577
S315080032942D03284358615969294003910399D9692B
S315080032A41143D961DB691A400492049B0022002168
S315080032B405204042FFF7A2F80022002102204042DE
S315080032C4FFF79CF80022002101204042FFF796F8F8
S315080032D480239B000593069400250795089505A960
S315080032E40948FFF7EFF80C2305930A3B069307955D
S315080032F401330893099405A99020C005FFF7E2F85D
S315080033040BB030BD00100240000800480D48854641
S315080033140D480E490E4A002302E0D458C45004331B
S31508003324C4188C42F9D30B4A0B4C002301E01360F2
S315080033340432A242FBD3FFF72BFF00F02DF8FFF768
S3150800334487FFFEE700200020C0000020C4000020FC
S315080033543C340008C4000020A4010020FEE710B590
S31508003364FFF782FCFA218900FEF7CEFEFFF778F80C
S315080033740420FFF791F80022002101204042FFF7BC
S315080033843DF810BD10B5FFF733F810BD10B5FFF7BB
S3150800339427F8FFF792F810BD70B500260C4D0D4CB2
S315080033A4641BA410A64209D1002600F019F80A4D98
S315080033B40A4C641BA410A64205D170BDB300EB5891
S315080033C498470136EEE7B300EB5898470136F2E71B
S315080033D43434000834340008343400083834000817
S315080033E4F8B5C046F8BC08BC9E467047F8B5C04652
S30D080033F4F8BC08BC9E467047B0
S315080033FC02030405060708090A0B0C0D0E0F10101C
S3150800340C0102030405060708090A0B0C0D0E0F101A
S3150800341C000000000000000001020304060708096A
S30D0800342C000000000102030480
S30908003434ED20000871
S30908003438C520000895
S3090800343C00127A00F2
S70508003311AE
